:020000040000FA
:1000000083169F01FC30850010308B0081139516FC
:1000100015158312073099000230A00085009F015A
:1000200005082039831601138312A101851A2114B2
:100030000230A000850005088B10630021183028CD
:10004000013085000000023085003F203F203F2026
:1000500000000000000005080439031920281828B2
:100060000130850000000000023085003F203F2065
:100070003F203F20050804390319302818280800BC
:10008000493452342034523465346D346F3474340E
:1000900065342034523465347034653461347434DA
:1000A000653472342E3420345034653474346534FD
:1000B00020344734723469346634663469347434B5
:1000C00068347334203432343034303434342034AF
:1000D0002D34523465346D346F34743465344534A2
:0E00E00078342D3434342E34613473346D345E
:02400E00C43CB0
:00000001FF
